:020000040000FA
:0400000034EF00F0E9
:100018005680D8CF04F0E8CF05F0E0CF06F0D9CF6E
:1000280007F0DACF08F0F2BAF2A405D0D59E08ECB2
:1000380007F0F29409D0F0B6F0A006D0000ED76E03
:10004800830ED66ED58EF09008C0DAFF07C0D9FFB0
:1000580006C0E0FF05C0E8FF04C0D8FF56901000B6
:1000680042EF10F00B500C10D8B402D0000E01D0A3
:10007800010E0F6E5550D8B44BD008D1700E09241C
:10008800D96E000E0A20DA6E0FB003D00001DF9897
:1000980002D00001DF881200F10E0924096EFF0E5C
:1000A8000A200A6E700E0924D96E000E0A20DA6E34
:1000B8000FB003D00001DF9A02D00001DF8A1200DE
:1000C800E20E0924096EFF0E0A200A6E700E09243A
:1000D800D96E000E0A20DA6E0FB003D00001DF9C43
:1000E80002D00001DF8C1200D30E0924096EFF0E26
:1000F8000A200A6E700E0924D96E000E0A20DA6EE4
:100108000FB003D00001DF9E02D00001DF8E120085
:1001180009C00DF00AC00EF00E50000AD8A4120053
:100128000D50000AD8B4AAD7010AD8B4A7D7030A31
:10013800D8B4A4D7010AD8B4A1D7070AD8B49ED78F
:10014800010AD8B49BD7030AD8B498D7010AD8B4FF
:1001580095D70F0AD8B492D7010AD8B48FD7030A13
:10016800D8B48CD7010AD8B489D7070AD8B486D7A7
:10017800010AD8B483D7030AD8B480D7010AD8B4FF
:100188008BD71F0AD8B488D7010AD8B485D7030AF1
:10019800D8B482D7010AD8B47FD7070AD8B47CD795
:1001A800010AD8B479D7030AD8B476D7010AD8B4E3
:1001B80073D70F0AD8B470D7010AD8B46DD7030A19
:1001C800D8B46AD7010AD8B467D7070AD8B464D7AD
:1001D800010AD8B461D7030AD8B472D7010AD8B4CF
:1001E8006FD73F0AD8B46CD7010AD8B469D7030AC5
:1001F800D8B466D7010AD8B463D7070AD8B460D789
:10020800010AD8B45DD7030AD8B45AD7010AD8B4BA
:1002180057D70F0AD8B454D7010AD8B451D7030A0C
:10022800D8B44ED7010AD8B44BD7070AD8B448D7A0
:10023800010AD8B459D7030AD8B456D7010AD8B492
:1002480053D71F0AD8B450D7010AD8B44DD7030AD8
:10025800D8B44AD7010AD8B447D7070AD8B444D77C
:10026800010AD8B441D7030AD8B43ED7010AD8B492
:100278003BD70F0AD8B438D7010AD8B435D7030A00
:10028800D8B432D7010AD8A412002ED75504D8A45E
:100298001200A0D1600E0924D96E000E0A20DA6E71
:1002A8000FB003D00001DF9802D00001DF881200F0
:1002B800FD0E0924096EFF0E0A200A6E600E09243D
:1002C800D96E000E0A20DA6E0FB003D00001DF9A53
:1002D80002D00001DF8A1200FA0E0924096EFF0E0F
:1002E8000A200A6E600E0924D96E000E0A20DA6E02
:1002F8000FB003D00001DF9C02D00001DF8C120098
:10030800F70E0924096EFF0E0A200A6E600E0924F2
:10031800D96E000E0A20DA6E0FB003D00001DF9EFE
:1003280002D00001DF8E120009C00DF00AC00EF0E5
:100338000E50000AD8A412000D50000AD8B4AAD74B
:10034800010AD8B4A7D7030AD8B4A4D7010AD8B4E5
:10035800AFD7070AD8B4ACD7010AD8B4A9D7030ACB
:10036800D8B4BAD7010AD8B4B7D70F0AD8B4B4D713
:10037800010AD8B4C5D7030AD8B4C2D7010AD8A489
:100388001200BED7F90E95D7F20EA7D7EB0EB9D744
:1003980009C00DF00AC00EF00E50000AD8A41200D1
:1003A8000D50000AD8B476D7010AD8B473D7030A17
:1003B800D8B470D7010AD8B46DD7070AD8B46AD7A9
:1003C800010AD8B467D7030AD8B464D7010AD8B4E5
:1003D800D9D70F0AD8B4D6D7010AD8B4D3D7030AC5
:1003E800D8B4D0D7010AD8B4CDD7070AD8B4CAD759
:1003F800010AD8B4C7D7030AD8B4C6D7010AD8B4F3
:10040800C3D71F0AD8B4C0D7010AD8B4BDD7030AC6
:10041800D8B4BAD7010AD8B4B7D7070AD8B4B4D76A
:10042800010AD8B4B3D7030AD8B4B0D7010AD8B4EC
:10043800ADD70F0AD8B4AAD7010AD8B4A7D7030AE8
:10044800D8B4A4D7010AD8A41200A0D7F10E31D786
:10045800E20E43D7D30E55D709C00DF00AC00EF0EF
:100468000E50000AD8A412000D50000AD8B412D7B2
:10047800010AD8B40FD7030AD8B40CD7010AD8B4E4
:1004880009D7070AD8B406D7010AD8B403D7030A8C
:10049800D8B400D7010AD8B4FDD60F0AD8B4FAD612
:1004A800010AD8B4F7D6030AD8B4F4D6010AD8B4E6
:1004B800F1D6070AD8B4EED6010AD8B4EBD6030AA7
:1004C800D8B4E8D6010AD8B4C1D71F0AD8B4BED761
:1004D800010AD8B4BBD7030AD8B4B8D7010AD8B42C
:1004E800B5D7070AD8B4B2D7010AD8B4AFD7030A28
:1004F800D8B4ACD7010AD8B4A9D70F0AD8B4A6D7AC
:10050800010AD8B4A3D7030AD8B4A0D7010AD8B42B
:100518009DD7070AD8B49AD7010AD8B497D7030A3F
:10052800D8B496D7010AD8B493D73F0AD8B490D78D
:10053800010AD8B48DD7030AD8B48AD7010AD8B427
:1005480087D7070AD8B484D7010AD8B481D7030A51
:10055800D8B47ED7010AD8B47BD70F0AD8B478D7D5
:10056800010AD8B475D7030AD8B472D7010AD8B427
:100578006FD7070AD8B46CD7010AD8B46BD7030A67
:10058800D8B468D7010AD8B465D71F0AD8B462D7D7
:10059800010AD8B45FD7030AD8B45CD7010AD8B423
:1005A80059D7070AD8B456D7010AD8B453D7030A7B
:1005B800D8B450D7010AD8B44DD70F0AD8B44AD7FF
:1005C800010AD8B447D7030AD8B444D7010AD8A433
:1005D800120040D75450010AD8B4A6D6030AD8B49A
:1005E800D7D6010AD8A4120037D7190E256E000EE7
:1005F800266E0AD2250E2E18D8B409D015C0D9FFF8
:1006080016C0DAFF2EC0DFFF154A162AFDD1000EEC
:100618002D6E000E2C6E000E2B6E03D02B84174A05
:10062800182A17C0F6FF18C0F7FF0800F550300A5F
:10063800D8B4F4D717C0F6FF18C0F7FF0800F55074
:10064800A5EC12F0D8A0ACD0000E2D6E000E2C6ECA
:100658002CC009F02DC00AF0000E0C6E0A0E0B6EAD
:1006680092EC12F009C02CF00AC02DF0D00E1D6ECD
:10067800FF0E1E6E17C0F6FF18C0F7FF0800F550F2
:100688001F6E206A1D501F261E5020221F502C2628
:1006980020502D22174A182A17C0F6FF18C0F7FF56
:1006A8000800F550A5EC12F0D8A07AD0D1D72B8E3F
:1006B80091D025C0D9FF26C0DAFFDECF23F0DDCFE9
:1006C80024F0020E2526000E262223502410D8A43A
:1006D80004D0E80E236E7F0E246E000E286E000EE6
:1006E800276E02D0274A282A275023241D6E285017
:1006F80024201E6E1DC0F6FF1EC0F7FFF86A050E07
:10070800F76403D00800F55005D0F6CFE1FFF7CF26
:10071800E2FFE7500009D8A4E5D72C50275C2D50FC
:100728002858D8B005D027502C5E28502D5A0DD007
:10073800000E2D6E000E2C6E08D015C0D9FF16C005
:10074800DAFF200EDF6E154A162A2C06D8A02D06D1
:100758002C28F3E12D28D8B41AD0EFD723C0F6FF00
:1007680024C0F7FFF86A15C0D9FF16C0DAFF050ED6
:10077800F76403D00800F55005D0F6CFE1FFF7CFB6
:10078800E2FFE750DF6E234A242A154A162A270675
:10079800D8A028062728E2E12828D8B435D1DED702
:1007A80017C0F6FF18C0F7FF174A182A0800F5CF38
:1007B8002EF02E50000AD8B433D1640AD8B40AD027
:1007C8000D0AD8B407D01A0AD8B473D70B0AD8B40C
:1007D8006ED71AD12BBE15D025C0D9FF26C0DAFF97
:1007E800DECF29F0DDCF2AF0020E2526000E2622C4
:1007F8002AAE44D0030E2B12296C2A1ED8B02A2AFE
:100808003DD025C0D9FF26C0DAFFDECF29F0DDCFE5
:100818002AF0020E2526000E262230D0010E2E6E5A
:100828002E50020D210EF324F66E7D0EF420F76E85
:100838000900F550295C0900F5502A58D8A026D09F
:100848002E2A050E2E18D8B421D0EAD7010E2E6E06
:100858002E50020D2B0EF324F66E7D0EF420F76E4B
:100868000900F550295C0900F5502A58D8A00ED087
:100878002E2A040E2E18D8B409D0EAD72B50800B94
:10088800000AD8B4CBD7800AD8B4E0D72C502D10A2
:10089800D8B409D02BC01DF0030E1D16D8B403D050
:1008A8002C06D8A02D062E501D6E1E6A2C501D5CDD
:1008B8001E50800A1F6E2D50800A1F58D8B005D0D0
:1008C8002E502C5E000E2D5A04D0000E2D6E000EF8
:1008D8002C6E2BA41ED02BC01DF0030E1D16D8B4F1
:1008E80008D015C0D9FF16C0DAFF2D0EDF6E154AE5
:1008F800162A2C502D10D8B42DD015C0D9FF16C0EB
:10090800DAFF300EDF6E154A162A2C06D8A02D06FF
:10091800F0D72C502D10D8B40FD015C0D9FF16C061
:10092800DAFF200EDF6E154A162A2C06D8A02D06EF
:100938002C502D10D8A4F1D72BC01DF0030E1D1676
:10094800D8B408D015C0D9FF16C0DAFF2D0EDF6E57
:10095800154A162A2EC022F053D02250020D210E1D
:10096800F324F66E7D0EF420F76E0900F5CF0BF038
:100978000A00F5CF0CF029C009F02AC00AF0D8EC1B
:1009880010F009C010F00AC011F0000E136E0A0E24
:10099800126E95EC11F01050300F2E6E29D029C030
:1009A80009F02AC00AF02250020D2B0EF324F66E2D
:1009B8007D0EF420F76E0900F5CF0BF00A00F5CF95
:1009C8000CF0D8EC10F009500F0B216E100E2124FA
:1009D800F66EF76A7F0EF7220800F5CF2EF008D0E2
:1009E8002B50800B000AD8B4B8D7800AD8B4D7D710
:1009F80015C0D9FF16C0DAFF2EC0DFFF154A162A28
:100A080022062228D8A4ECD717C0F6FF18C0F7FF93
:100A1800174A182A0800F5CF2EF02E50D8A4EAD588
:100A280015C0D9FF16C0DAFF000EDF6E1200E3C052
:100A38003DF0E4C03EF0E5C03FF0E6C040F0000EF7
:100A4800426E020E0D6E3D50B6EC11F0F3EC0EF056
:100A5800416EB7D14250D8B402D04206BFD1010E80
:100A6800416EBCD1030E426002D0422AB7D1000EBB
:100A7800426EB4D15350020D490EF324D96E000EC4
:100A8800F420DA6EDECF38F0DDCF39F0100E3826DC
:100A9800000E392239BE03D03904D8B00CD05350D7
:100AA800020D490EF324D96E000EF420DA6E100EF2
:100AB800DE26000EDD225350020D490EF324D96EB6
:100AC800000EF420DA6E5350020D430EF324E16E4B
:100AD800000EF420E26EDE50E65CE650800A3C6EC2
:100AE800DE50800A3C58D8B079D15350020D490ED7
:100AF800F324D96E000EF420DA6E5350020D430E23
:100B0800F324E16E000E0FD15350020D490EF32469
:100B1800D96E000EF420DA6EDECF38F0DDCF39F072
:100B2800010E3826000E392239BE03D03904D8B058
:100B38000BD05350020D490EF324D96E000EF42049
:100B4800DA6EDE2A000EDD225350020D490EF32420
:100B5800D96E000EF420DA6E5350020D430EF324C2
:100B6800E16E000EF420E26EDE50E65CE650800A8C
:100B78003C6EDE50800A3C58D8A0B7D72FD15350CE
:100B8800020D430EF324D96E000EF420DA6EDECF88
:100B980038F0DDCF39F0100E3826000E392239BE74
:100BA80003D03904D8B01AD15350020D430EF324A0
:100BB800D96E000EF420DA6E100EDE261ED05350C9
:100BC800020D430EF324D96E000EF420DA6EDECF48
:100BD80038F0DDCF39F0010E3826000E392239BE43
:100BE80003D03904D8B0FAD05350020D430EF32481
:100BF800D96E000EF420DA6EDE2A000E2CD0425098
:100C0800000AD8B437D7010AD8B47ED7030AD8B4B3
:100C1800B6D7010AD8B4D3D7E1D05350020D490E44
:100C2800F324D96E000EF420DA6EDECF38F0DDCF73
:100C380039F0F00E3824FF0E3920800BD8A4CED01E
:100C48005350020D490EF324D96E000EF420DA6ECB
:100C5800F00EDE26FF0EDD22C1D05350020D490EE4
:100C6800F324D96E000EF420DA6EDECF38F0DDCF33
:100C780039F0FF0E3824FF0E3920800BD8A4AED0EF
:100C88005350020D490EF324D96E000EF420DA6E8B
:100C9800DE06000EDD5AA2D05350020D430EF32497
:100CA800D96E000EF420DA6EDECF38F0DDCF39F0E1
:100CB800F00E3824FF0E3920800BD8A40CD05350E6
:100CC800020D430EF324D96E000EF420DA6EF00EF6
:100CD800DE26FF0EDD225350020D490EF324D96E95
:100CE800000EF420DA6E5350020D430EF324E16E29
:100CF800000EF420E26EDE50E65CE650800A3C6EA0
:100D0800DE50800A3C58D8B069D05350020D430ECB
:100D1800F324D96E000EF420DA6E5350020D490EFA
:100D2800F324E16E000EF420E26EDECFE6FFDDCFA5
:100D3800E5FF54D05350020D430EF324D96E000E34
:100D4800F420DA6EDECF38F0DDCF39F0FF0E38242C
:100D5800FF0E3920800BD8A40BD05350020D430E40
:100D6800F324D96E000EF420DA6EDE06000EDD5A8A
:100D78005350020D490EF324D96E000EF420DA6E9A
:100D88005350020D430EF324E16E000EF420E26E80
:100D9800DE50E65CE650800A3C6EDE50800A3C5825
:100DA800D8A0B3D71BD04250000AD8B436D7010A0E
:100DB800D8B453D7030AD8B46FD7010AD8B4BAD76E
:100DC8000DD04150020AD8B445D6010AD8B417D775
:100DD800070AD8B4E8D7010AD8B444D655EC0BF0C2
:100DE800020E0D6E3D0E4224D96EDA6A000EDA222A
:100DF800DF50B6EC11F04104D8A428D6020E0D6ECF
:100E0800000EB6EC11F0120000018D51016E8E51EA
:100E1800026E8D4B8E2B025004E1650E015CD8A04A
:100E280012D0000E8E6F000E8D6F8CAE02D0010EA8
:100E380001D0000EFF0A016E013201328C500118F8
:100E48007F0B01188C6E000E52D08B80898C898E96
:100E58008D80898403A002D08D8201D08D9203A257
:100E680002D08D8001D08D9003A402D0898A01D050
:100E7800899A03A602D0898601D089960A0EE82E9F
:100E8800FED700D08994700E0324D96EDA6A000E5A
:100E9800DA220001DFA802D08D8001D08D90700E7B
:100EA8000324D96EDA6A000EDA220001DFAA02D022
:100EB800898E01D0899E700E0324D96EDA6A000EDD
:100EC800DA220001DFAC02D0898C01D0899C700E37
:100ED8000324D96EDA6A000EDA220001DFAE02D0EE
:100EE8008B8001D08B90040EE82EFED70328036E6A
:100EF8000E0E0364AAD78B80898C898E8D80898495
:100F08008986898A8D808D820A0EE82EFED700D0C8
:100F180089948B90899C899E8D902FD1000E48D002
:100F28008B80898C898E8D80899203A002D08D82D6
:100F380001D08D9203A202D08D8001D08D900A0E2F
:100F4800E82EFED700D08982700E0324D96EDA6AA3
:100F5800000EDA220001DFA802D08D8001D08D902A
:100F6800700E0324D96EDA6A000EDA220001DFAAB5
:100F780002D0898E01D0899E700E0324D96EDA6A58
:100F8800000EDA220001DFAC02D0898C01D0899CE6
:100F9800700E0324D96EDA6A000EDA220001DFAE81
:100FA80002D08B8001D08B90040EE82EFED7032848
:100FB800036E020E0364B4D78B80898C898E8D8072
:100FC80089928D808D820A0EE82EFED700D0898204
:100FD8008B90899C899E8D901200000E4DD08B803D
:100FE800898C898E8D80899203A002D08D8201D050
:100FF8008D9203A202D08D8001D08D9003A402D0DF
:10100800898A01D0899A0A0EE82EFED700D08982F3
:10101800700E0324D96EDA6A000EDA220001DFA806
:1010280002D08D8001D08D90700E0324D96EDA6ABB
:10103800000EDA220001DFAA02D0898E01D0899E33
:10104800700E0324D96EDA6A000EDA220001DFACD2
:1010580002D0898C01D0899C700E0324D96EDA6A7B
:10106800000EDA220001DFAE02D08B8001D08B9017
:10107800040EE82EFED70328036E060E0364AFD7CE
:101088008B80898C898E8D808992898A8D808D82CA
:101098000A0EE82EFED700D089828B90899C899E03
:1010A8008D901200000E52D08B80898C898E8D8095
:1010B800898203A002D08D8201D08D9203A202D032
:1010C8008D8001D08D9003A402D0898A01D0899A9D
:1010D80003A602D0898601D089960A0EE82EFED78B
:1010E80000D08992700E0324D96EDA6A000EDA22D3
:1010F8000001DFA802D08D8001D08D90700E0324EE
:10110800D96EDA6A000EDA220001DFAA02D0898ECF
:1011180001D0899E700E0324D96EDA6A000EDA2295
:101128000001DFAC02D0898C01D0899C700E0324A9
:10113800D96EDA6A000EDA220001DFAE02D08B80A7
:1011480001D08B90040EE82EFED70328036E0E0EF6
:101158000364AAD78B80898C898E8D808982898641
:10116800898A8D808D820A0EE82EFED700D089925A
:101178008B90899C899E8D9012005450010AD8B496
:10118800CDD6030AD8B429D7010AD8A412008AD721
:10119800D388D38AD38CD396FC0ED3169B9C000E8F
:1011A8000F01386F000E896E100E926E000E396FA7
:1011B800020E936E000E3A6F000E8B6EC00E946E88
:1011C800000E3B6F000E956E000E3C6F000E966E83
:1011D8009E969D86F28EF28C9F86D08EF28CF28E31
:1011E800F28AF194000ED76E830ED66ED58ED58C0A
:1011F800D59AD596D550F80B0509D56EF28AF29492
:10120800F19AF09CF090F086000E0001FD6F000E40
:10121800FC6F600EFC25D96E000EFD21DA6EFF0E04
:10122800DF6E700EFC25E16E000EFD21E26EDFCF51
:10123800E7FFFC4BFD2BFDBFECD7FD5104E1100E81
:10124800FC5DD8A0E6D78B828B848B868C808C94AF
:10125800899289948C868B888B8A8C828986898AE4
:101268008D808D828B80898C898E8D808C8E79EC97
:1012780010F0010E72EC11F00F0E72EC11F0900EDE
:10128800156E000E166EFE0E176E7E0E186EFB0E95
:10129800196E7F0E1A6EF9EC02F0000E0D6E000E3C
:1012A800B6EC11F0900E0D6E000E0E6ED4EC11F02F
:1012B800010E0D6E000EB6EC11F0650E0D6E7F0E70
:1012C8000E6ED4EC11F0020E0D6E000EB6EC11F09D
:1012D800D50E0D6E7F0E0E6ED4EC11F0030E0D6E52
:1012E800000EB6EC11F0EB0E0D6E7E0E0E6ED4EC09
:1012F80011F0030E0D6E070EB6EC11F001D000F0E0
:10130800F3EC0EF0E806D8A4FAD755EC0BF094D01D
:1013180086EC0EF091D05250D8B402D05206F5D7D0
:10132800030E06D0030E526002D0522AEED7000EEA
:10133800526EEBD75350D8B402D05306E6D7020EFC
:1013480030D08A0E5324D96EDA6A000EDA22DF50C2
:10135800D8B408D08A0E5324D96EDA6A000EDA227D
:10136800DF06D3D78A0E5324D96EDA6A000EDA2242
:10137800EB0E5324E16EE26A000EE222E750000110
:10138800F56FF50544D05250000AD8B4D3D7010AF6
:10139800D8B4D7D751D0020E536002D0532AB5D74C
:1013A800000E536EB2D7FF0E0001F56FFF0EF66FF9
:1013B800EB0E5324D96EDA6A000EDA22DF50F76F8B
:1013C800F86BF551F727F651F8238A0E5324D96E96
:1013D800DA6A000EDA22DF50F96FFA6BF751F95D1D
:1013E800FA51800AFB6FF851800AFB59D8B008D02F
:1013F8008A0E5324D96EDA6A000EDA22DF2A85D7DC
:101408008A0E5324D96EDA6A000EDA22000EDF6ED5
:101418007CD71BEC05F010D06AEC12F00DD05250BE
:10142800000AD8B4B8D7010AD8B4BDD7030AD8B4CB
:10143800F0D7010AD8B4F0D7F3EC0EF0010AD8B40B
:1014480067D7030AD8B49FD7010AD8B464D7070A64
:10145800D8B468D7010AD8B4E2D7EED7010E72EC37
:1014680011F00F0E72EC11F0000E0D6E000EB6ECBE
:1014780011F0630E0D6E7E0E0E6ED4EC11F0010E9F
:101488000D6E000EB6EC11F0BB0E0D6E7D0E0E6EDD
:10149800D4EC11F0020E0D6E000EB6EC11F0E50E54
:1014A8000D6E7D0E0E6ED4EC11F010D0000E556E40
:1014B80020D0010E556E010E07D0010E556E020E9A
:1014C80003D0010E556E030E546E13D08A0E5324AA
:1014D800D96EDA6A000EDA22DF50000AD8B4E6D7ED
:1014E800010AD8B4E6D7030AD8B4E7D7010AD8B4B2
:1014F800E8D75350020D490EF324D96E000EF4209C
:10150800DA6EDECF32F0DDCF33F03BD0030E0D6E56
:10151800000EB6EC11F0900E156E000E166E330E1E
:10152800176E7D0E186E5350020D490EF324D96EB6
:10153800000EF420DA6EDECF19F0DDCF1AF053502A
:10154800020D430EF324D96E000EF420DA6EDECFBE
:101558001BF0DDCF1CF0F9EC02F0900E0D6E000EC2
:101568000E6ED4EC11F0FF0E3224096EFF0E3320FC
:101578000A6E000E0C6E010E0B6E36EC00F0324A4D
:10158800332A5350020D430EF324D96E000EF42073
:10159800DA6E3250DE5CDE50800A316E3350800ADB
:1015A8003158D8B0B3D74FC009F050C00AF0000E78
:1015B8000C6E0A0E0B6E92EC12F009C00FF00AC006
:1015C80010F029EC11F05350020D490EF324D96E96
:1015D800000EF420DA6EDECF32F0DDCF33F03BD0F0
:1015E800030E0D6E000EB6EC11F0900E156E000E87
:1015F800166E4B0E176E7D0E186E5350020D490E67
:10160800F324D96E000EF420DA6EDECF19F0DDCFA8
:101618001AF05350020D430EF324D96E000EF42035
:10162800DA6EDECF1BF0DDCF1CF0F9EC02F0900E85
:101638000D6E000E0E6ED4EC11F0FF0E3224096E02
:10164800FF0E33200A6E000E0C6E000E0B6E36EC89
:1016580000F0324A332A5350020D430EF324D96E58
:10166800000EF420DA6E3250DE5CDE50800A316EF5
:101678003350800A3158D8B0B3D74FC009F050C0A2
:101688000AF0000E0C6E0A0E0B6E92EC12F009C0F6
:101698000FF00AC010F029EC11F00009D8A41200CC
:1016A80028D75350020DDD0EF324D96E000EF42016
:1016B800DA6EDECF30F0DDCF31F0000E156E010EA0
:1016C800166E7B0E176E7D0E186E5350020D490E66
:1016D800F324D96E000EF420DA6EDECF19F0DDCFD8
:1016E8001AF05350020D430EF324D96E000EF42065
:1016F800DA6EDECF1BF0DDCF1CF0F9EC02F0000E45
:10170800326E010E336EAE0E366E000E376E6DD031
:101718008A0E5324D96EDA6A000EDA22DF502F6E51
:101728002F50020DD50EF324D96E000EF420DA6E78
:10173800DECF34F0DDCF35F0AE0E156E000E166E2E
:10174800DF0E176E7F0E186E4FC019F050C01AF0DA
:10175800F9EC02F0AE0E366E000E376E50D08A0EDF
:101768005324D96EDA6A000EDA22DF502F6E2F501A
:10177800020DC30EF324D96E000EF420DA6EDECF0C
:1017880034F0DDCF35F0AE0E156E000E166EDF0E9E
:10179800176E7F0E186EF0C019F0F1C01AF0F9EC50
:1017A80002F0D8D78A0E5324D96EDA6A000EDA22EC
:1017B800DF502F6E2F50020DE70EF324D96E000E66
:1017C800F420DA6EDECF34F0DDCF35F0AE0E156ED4
:1017D800000E166EDF0E176E7F0E186EEEC019F033
:1017E800EFC01AF0F9EC02F0B5D75350000AD8B49C
:1017F8008FD7010AD8B4B3D7030AD8B4D3D7010E08
:1018080072EC11F0900E156E000E166EF60E176E35
:101818007F0E186E30C019F031C01AF0F9EC02F0E2
:10182800000E0D6E000EB6EC11F0900E0D6E000E4F
:101838000E6ED4EC11F0900E156E000E166EF60EAC
:10184800176E7F0E186E34C019F035C01AF0F9EC17
:1018580002F0010E0D6E000EB6EC11F0900E0D6E3A
:10186800000E0E6ED4EC11F0900E156E000E166E72
:10187800F60E176E7F0E186E32C019F033C01AF0CC
:10188800F9EC02F0020E0D6E000EB6EC11F0900E9F
:101898000D6E000E0E6ED4EC11F0900E156E000E4B
:1018A800166EF60E176E7F0E186E36C019F037C01A
:1018B8001AF0F9EC02F0030E0D6E000EB6EC11F002
:1018C800900E0D6E000E0E6ED4EC11F052C00DF09D
:1018D800000EB6EC11F01200010E72EC11F00F0EB2
:1018E80072EC11F0000E0D6E000EB6EC11F0630EE6
:1018F8000D6E7D0E0E6ED4EC11F0010E0D6E000E05
:10190800B6EC11F0BB0E0D6E7D0E0E6ED4EC11F020
:10191800020E0D6E000EB6EC11F0E50E0D6E7D0E8A
:101928000E6ED4EC11F05350020D490EF324D96E0B
:10193800000EF420DA6EDECF34F0DDCF35F091D032
:10194800030E0D6E000EB6EC11F0900E156E000E23
:10195800166E4E0E176E7E0E186E34C019F035C016
:101968001AF0F9EC02F0900E0D6E000E0E6ED4EC2B
:1019780011F0030E0D6E0C0EB6EC11F050D03404BD
:1019880009EC12F0040E306E0C0E2F6E340EE82E99
:10199800FED72F2EFCD7302EFAD70F0E09EC12F0F7
:1019A8004BD0000E336E0E0E0FD0000E336E0D0EA0
:1019B8000BD0000E336E0B0E07D0000E336E070EE1
:1019C80003D0000E336E0F0E326E16D034C02FF0D7
:1019D80035C030F03050000AD8A4F3D72F50010A90
:1019E800D8B4DFD7030AD8B4E0D7010AD8B4E1D70E
:1019F800070AD8B4E2D7E5D7325022EC12F0110E1C
:101A0800306E3C0E2F6ECB0EE82EFED72F2EFCD755
:101A1800302EFAD700F0325022EC12F00DD08A0E98
:101A28005324D96EDA6A000EDA22DF50000AD8B4DD
:101A3800A6D7010AD8B4CAD7EEC009F0EFC00AF099
:101A4800000E0C6E0A0E0B6E92EC12F009C00FF02D
:101A58000AC010F029EC11F00009D8A41200344A89
:101A6800352A5350020D430EF324D96E000EF4208C
:101A7800DA6E3450DE5CDE50800A316E3550800AF2
:101A88003158D8A050D75CD7010E72EC11F00F0E68
:101A980072EC11F0000E0D6E000EB6EC11F0240E73
:101AA8000D6E7E0E0E6ED4EC11F0010E0D6E000E52
:101AB800B6EC11F0BB0E0D6E7D0E0E6ED4EC11F06F
:101AC800020E0D6E000EB6EC11F0E50E0D6E7D0ED9
:101AD8000E6ED4EC11F05350020D490EF324D96E5A
:101AE800000EF420DA6EDECF32F0DDCF33F071D0A5
:101AF800030E0D6E000EB6EC11F0900E156E000E72
:101B0800166E540E176E7F0E186E32C019F033C061
:101B18001AF0F9EC02F0900E0D6E000E0E6ED4EC79
:101B280011F0030E0D6E0C0EB6EC11F01BD0320442
:101B380009EC12F0070E306E170E2F6E6A0EE82EA3
:101B4800FED72F2EFCD7302EFAD700D00F0E09EC77
:101B580012F02AD0325051EC0FF026D0325000EC5F
:101B68000EF022D08A0E5324D96EDA6A000EDA22D9
:101B7800DF50000AD8B4DBD7010AD8B4EBD7030A80
:101B8800D8B4E8D7010AD8B4E5D7070AD8B4E6D755
:101B9800010AD8B4E3D7030AD8B4E0D7010AD8B405
:101BA800DDD70F0AD8B4DAD7F0C009F0F1C00AF0CF
:101BB800000E0C6E0A0E0B6E92EC12F009C00FF0BC
:101BC8000AC010F029EC11F00009D8A41200324A1A
:101BD800332A5350020D430EF324D96E000EF4201D
:101BE800DA6E3250DE5CDE50800A316E3350800A85
:101BF8003158D8A070D77CD7096E09C012F0000EF2
:101C080012B0010E0A6E000E12B2010E0B6E000E1B
:101C180012B4010E0C6E000E12B6010E0D6E000EFF
:101C280012B8010E0E6E000E12BA010E0F6E000EE3
:101C380012BC010E106E000E12BE010E116EF29E45
:101C48008CA405D08B828B848B868C808C94350EEB
:101C5800E82EFED700F05104D8A404D0210EE82EB7
:101C6800FED700F08C841D0EE82EFED700F00AB0D7
:101C780002D08C9001D08C800BB002D08B9601D012
:101C88008B860CB002D08B9401D08B840DB002D01F
:101C98008B9201D08B829D0EE82EFED700F0510466
:101CA800D8A404D0210EE82EFED700F00EB002D042
:101CB8008C9001D08C800FB002D08B9601D08B868F
:101CC80010B002D08B9401D08B8411B002D08B92CB
:101CD80001D08B82680EE82EFED75150D8A407D0C9
:101CE800FB0E00D000D0E82EFCD700D000F0F28E1A
:101CF8008B828B848B868C80060EE82EFED700D0D4
:101D08008C941200010E72EC11F00F0E72EC11F0AF
:101D1800000E0D6E000EB6EC11F0A60E0D6E7D0EC7
:101D28000E6ED4EC11F0010E0D6E000EB6EC11F033
:101D380015D0FA0E0D6E7D0E0E6ED4EC11F018D083
:101D48000F0E0D6E7E0E0E6ED4EC11F011D0390E02
:101D58000D6E7E0E0E6ED4EC11F00AD05350000AB0
:101D6800D8B4E7D7010AD8B4EBD7030AD8B4EFD769
:101D7800020E0D6E000EB6EC11F0D00E0D6E7D0E3B
:101D88000E6ED4EC11F0030E0D6E000EB6EC11F0D1
:101D9800910E0D6E7D0E0E6ED4EC11F0000E0D6ED0
:101DA800070EB6EC11F0F3EC0EF0E806D8B40CD040
:101DB80055EC0BF0120032EC0AF0FAD748EC0DF0B3
:101DC800F7D770EC0CF0F4D75350000AD8B4F3D717
:101DD800010AD8B4F3D7030AD8B4F3D7E9D78C8863
:101DE8008C9A8C9C340E0D6EF20EE82EFED70D2EBA
:101DF800FCD7000E80B8010E0E6E0EC009F0010E61
:101E0800ABEC10F00009D8B402D0010E1200000E9D
:101E180082BC010E0E6E0EC009F0020EABEC10F083
:101E28000009D8B402D0020E1200000E82BE010EC4
:101E38000E6E0EC009F0050EABEC10F00009D8B418
:101E480002D0050E12008C988C8A8C9C340E0D6E74
:101E5800F20EE82EFED70D2EFCD7000E80B8010E2C
:101E68000E6E0EC009F0030EABEC10F00009D8B4EA
:101E780002D0030E1200000E82BC010E0E6E0EC0C0
:101E880009F0040EABEC10F00009D8B402D0040E2F
:101E980012008C988C9A8C9CA2D70A6E0AC00FF0FC
:101EA800000E0FB0010E0B6E000E0FB2010E0C6E7D
:101EB800000E0FB4010E0D6E000E0FB6010E0E6E61
:101EC800F29E8CA405D08B828B848B868C808C941C
:101ED800DD0EE82EFED700F08C84280EE82EFED703
:101EE8000BB002D08C9001D08C800CB002D08B96B5
:101EF80001D08B860DB002D08B9401D08B840EB0AC
:101F080002D08B9201D08B82F28E5E0E096E800E0B
:101F1800E82EFED7092EFCD700D08B828B848B86C7
:101F28008C801200030E0D6E040EB6EC11F0F3EC6B
:101F38000EF0386E1BD0010E386E23D00001F1BFB1
:101F480006D0F1511EE1090EF05DD8B01AD0F04B61
:101F5800F12B17D00001F1BF14D0F15103E1F005C6
:101F6800D8A00FD0F007D8A0F1070BD03850020A3C
:101F7800D8B4E1D7010AD8B4E1D7070AD8B4EAD768
:101F8800010A55EC0BF03804D8A4D1D7030E0D6E16
:101F9800000EB6EC11F01200030E0D6E040EB6EC36
:101FA80011F0F3EC0EF0386E1BD0010E386E23D012
:101FB8000001EFBF06D0EF511EE1090EEE5DD8B06B
:101FC8001AD0EE4BEF2B17D00001EFBF14D0EF5112
:101FD80003E1EE05D8A00FD0EE07D8A0EF070BD08D
:101FE8003850020AD8B4E1D7010AD8B4E1D7070AB1
:101FF800D8B4EAD7010A55EC0BF03804D8A4D1D7E5
:10200800030E0D6E000EB6EC11F01200030E0D6EED
:10201800040EB6EC11F0F3EC0EF0386E19D0010E88
:10202800386E21D050BE06D050501DE1090E4F5CCD
:10203800D8B019D04F4A502A16D050BE14D050509C
:1020480003E14F04D8A00FD04F06D8A050060BD0FC
:102058003850020AD8B4E3D7010AD8B4E3D7070A3C
:10206800D8B4EBD7010A55EC0BF03804D8A4D3D771
:10207800030E0D6E000EB6EC11F01200E00EF66EB7
:10208800230EF76E000EF86E00EEC3F010EE32F07D
:102098000900F5CFEEFFE550E150FAE1680EF66E63
:1020A800250EF76E000EF86E00EE43F010EE0FF0FE
:1020B8000900F5CFEEFFE550E150FAE101EE00F03E
:1020C800150EEE6AE806FDE100EE60F0630EEE6ABA
:1020D800E806FDE1556A546A536A526A5690569268
:1020E800000EF86E0001CCEF08F081908194819683
:1020F800960E01EC11F0300E3AEC12F000D000D040
:10210800BCEC12F0290E01EC11F0BCEC12F0010E3F
:1021180001EC11F0BCEC12F052EC12F0200E3AEC8B
:1021280012F000D000D0BCEC12F052EC12F0010E0C
:1021380072EC11F0280E72EC11F0080E72EC11F02E
:10214800060E72EC11F00C0E72EC11F012000C6E0F
:10215800800E0C24D96EDA6A000EDA220950DE18D5
:10216800D8B420D0030E0B6E080E0A6E770EE82E38
:10217800FED70A2EFCD70B2EFAD700F0800E0C24BF
:10218800D96EDA6A000EDA220950DE18D8B40AD0FD
:10219800800E0C24D96EDA6A000EDA2209C0DFFF3D
:1021A80009501200000E1200000E0F6E000E0E6E87
:1021B8000B500C10D8B41CD0010E0D6E04D0D89062
:1021C8000B360C360D2A0CAEFAD7D8900E360F36D1
:1021D8000B50095C0C500A58D8A005D00B50095E6A
:1021E8000C500A5A0E80D8900C320B320D2EEDD7B7
:1021F8000EC009F00FC00AF012000C6E000E0E6E31
:10220800000E0D6E14D0000E106E000E0F6E0D0E27
:10221800E82EFED700F00F4A102A10BEF8D710504B
:1022280004E10A0E0F5CD8A0F2D70D4A0E2A0C5012
:10223800096E0A6A09500D5C0E50800A0B6E0A502E
:10224800800A0B58D8B01200DED7000E146E000EAC
:10225800136E15D0030E126E080E116E770EE82E4F
:10226800FED7112EFCD7122EFAD700F07FEC12F011
:10227800E806D8A402D0010E1200134A142A0F50FF
:10228800135C1450800A116E1050800A1158D8A09F
:10229800E1D7000E12000C6E52EC12F00C50F00B4D
:1022A8000B6E0B503AEC12F0050EE82EFED700F03C
:1022B8008194818000D000D000D000D0BCEC12F016
:1022C8000C3A0C50F00B0B6E0B503AEC12F0050E5A
:1022D800E82EFED700F0BCEC12F012000C6E52ECA7
:1022E80012F00C50F00B0B6E0B503AEC12F0050E7E
:1022F800E82EFED700F08194819000D000D000D065
:1023080000D0BCEC12F00C3A0C50F00B0B6E0B50DA
:102318003AEC12F0050EE82EFED700F0BCEC12F0F5
:10232800120012501310D8B418D0010E146E04D035
:10233800D89012361336142A13AEFAD71250105CFE
:1023480013501158D8A004D01250105E1350115ACF
:10235800D89013321232142EF1D710C010F011C0D9
:1023680011F012000E6E130E0E6408D012000E8CBF
:1023780012D0140E01D0540E0E260DD00D50000AA6
:10238800D8B409D0010AD8B4F2D7030AD8B4F1D71F
:10239800010AD8B4F0D70E8E0E5072EC11F012006C
:1023A8000DC0F6FF0EC0F7FFF86A050EF76403D0FC
:1023B8000800F55005D0F6CFE1FFF7CFE2FFE75070
:1023C8000F6E06D00F504FEC11F00D4A0E2AE8D7C9
:1023D8000F50D8B41200F6D7EF7FB47F9E7FA97F45
:1023E800217F437F327F917F847FB27EC57ED87EF6
:1023F8009F7ECA7FBF7F757F090A11128B7E777E09
:1024080004090201000100960003096E09C00AF0E0
:102418008C940AA002D08C8001D08C900AA202D0A1
:102428008B8601D08B960AA402D08B8401D08B9422
:102438000AA602D08B8201D08B921200096E09C0C5
:102448000AF00AA002D08C8201D08C920AA202D093
:102458008B8A01D08B9A0AA402D08B8801D08B98E2
:102468000AA602D08C8601D08C961200096E09C08B
:102478000AF00AA802D0818801D081980AAA02D05D
:10248800818A01D0819A0AAC02D0818C01D0819CCA
:102498000AAE02D0818E01D0819E1200938E819067
:1024A8008184BCEC12F00D0EE82EFED700F0000E71
:1024B8008ABE010E096EBCEC12F00950D8A4EED702
:1024C8008194939E140EE82EFED7120009D00AECD0
:1024D80010F0120096EC0FF01200D0EC0FF0120082
:1024E8005350000AD8B4F3D7010AD8B4F3D7030A73
:1024F800D8A41200F2D78C888C9A8C9C340E096E62
:10250800F20EE82EFED7092EFCD7000E80B8010E79
:102518000A6E8C988C9A8C9C0A50120009500B02F7
:10252800F3CF0DF0F4CF0EF009500C02F3500E2645
:102538000A500B02F3500E260DC009F00EC00AF027
:1025480012000B6E000E0A6E3A0E0B6005D02F0EAD
:102558000B6402D0010E0A6E0AC009F0093012009D
:0F2568003C0010000F0001000100010001000104
:0C2578008186040EE82EFED7819612002A
:107D20000001000A006400E80310270100100000B1
:107D30000100106C616D7073202530327820746FF3
:107D40002025303278204F4E2020006C616D7073FA
:107D5000202530327820746F2025303278204F462D
:107D600046200020536F6C656E6F696420746573E4
:107D7000742072756E6E696E67200066726F6D3A60
:107D800030782530327820746F3A30782530327868
:107D90000020746F2063616E63656C2020202020BA
:107DA000202020202000207072657373204F4B200C
:107DB000746F202020202020202000207072657306
:107DC0007326686F6C64204F4B20202020202000F9
:107DD00020616E79206F74686572206B6579202050
:107DE000202020200020746F2063616E63656C206A
:107DF00074657374202020202000207374617274D5
:107E0000204C616D70205465737420202020002068
:107E1000737461727420536F756E6420546573744B
:107E20002020200020536F756E64207465737420C9
:107E300072756E6E696E67200020737461727420B3
:107E4000536F6C656E6F69642054657374002070A5
:107E5000756C736520736F6C656E6F696420253077
:107E6000327800204C616D702074657374207275D7
:107E70006E6E696E672000436F6E74696E6F757306
:107E800020536F6C656E6F696473004D6F6D656E26
:107E90007461727920536F6C656E6F696473003220
:107EA0006E642041532D323531382D32332836302F
:107EB00029003173742041532D323531382D32333E
:107EC0002836302900326E642041532D3235313846
:107ED0002D34332831322900326E642041532D3243
:107EE0003531382D353228323429002070726573CF
:107EF00073204F4B20746F20737461727400426161
:107F00006C6C79205465737465722056202573005B
:107F100030313233343536373839616263646566FF
:107F20000041532D323531382D35362028536F2BF3
:107F3000290041532D323531382D36312028532632
:107F400054290041532D323531382D3537202856EC
:107F50006F63290020706C617920736F756E6420E7
:107F600025303278002020207777772E6C6973795E
:107F70002E646576005465737420536F6C656E6F64
:107F80006964730043686561702053717565616B46
:107F90000053617920497420416761696E00415343
:107FA0002D323531382D35300041532D32353138B1
:107FB0002D35310041532D323531382D33320054B7
:107FC00065737420536F756E640054657374204C30
:107FD000616D707300202020205245414459007487
:107FE0003A25642073656300286E756C6C29004324
:107FF00068696D6573003E20257300302E320000E5
:020000040020DA
:08000000FFFFFFFFFFFFFFFF00
:020000040030CA
:0E000000FF281F3CFFBF85FF0FC00FE00F4021
:00000001FF
